:10000000CB280730831685008312850141309F007D
:10001000503083169F0074309100073087003F30C6
:1000200083128700853083168100FF23900083129E
:1000300090018B130800A1002108013A0319272819
:10004000033A03192B28013A03192F283328D130FA
:1000500083129F003628D53083129F003628D9306E
:1000600083129F003628093083129F0008000B1965
:1000700050288312851101082402031C8512831263
:1000800001082502031C8712831201082602031CA3
:10009000071283120108270203183728871137280F
:1000A0000B11831285168515FF3087000800A1000B
:1000B000A108031D5F2883121E08A8008F28831241
:1000C0001E0803196A281E0B6F28DC3083161E02D7
:1000D00003186F2828302107840080018F280330FF
:1000E00083121E0203187D281E08023A031D83286E
:1000F0001C3083161E02031C83282830210784002D
:10010000FF3080008F28DC3083161E02A2002830CA
:10011000210784000310220D80000310800D0800C9
:10012000A100A108031DA3282908A4002A0824026D
:1001300003189C282A08A4002B0824020318A228CC
:100140002B08A40008002808A200283021078400FA
:100150000008A30023082202031CB0282208A300E1
:1001600024302107840000082302031CBD2824300A
:100170002107840023088000080024302107840020
:10018000000803190800AC08031DCA282430210701
:100190008400800308000120AC012030AC07A001DE
:1001A000043020020318CD28372020081B203720D8
:1001B00083129F14372020085720372020089020D2
:0401C000A00AD02899
:0207FE003C3489
:084000000F000A00000001009E
:02400E00C521CA
:00000001FF
